:020000040000FA
:10000000283084005830A0008001840AA00B042806
:10001000103095002730960000308E0000308F00A1
:10002000013090000B30970007309F008316FF309F
:100030008500831283168630860083120C1D1E28CD
:100040000C116400A914A9182915A91C2911051956
:100050002A282911A9192D28291129192916291DFC
:100060002912A91E34282911291AA916291EA912F4
:10007000291D3F28291B3F28AA0F3F28AB0A291911
:100080002917291D291300302B0203194E28A0001F
:1000900020092B05A006A01B5328552801302A0251
:1000A000031C53285528291156282915A91F5928FA
:1000B000291129192C14291D2C10A9182915A91C3E
:1000C0002911AC1029192C15291D2C11AC196928DE
:1000D0002C112C1929162C1D29122C1E70282C11BC
:1000E000291A2C16291E2C122C1D7728AC1429191C
:1000F0002C15291D2C1105197E282C112C192916B7
:100100002C1D2912AC1E85282C11291AAC16291E6B
:10011000AC122C1D8C28AC14AC182915AC1C291160
:10012000291D97282C1B9728AD0F9728AE0A29194F
:100130002C17291D2C1300302E020319A628A0000D
:1001400020092E05A006A01BAB28AD2803302D02E8
:10015000031CAB28AD282911AE2829152919A9158A
:10016000291DA911A9182915A91C2911AC1BB928E9
:100170002911291DD5282F18D528AD0FC028AE0A62
:1001800000302E020319CB28A00020092E05A0065E
:10019000A01BD028D12801302D02031CD028D12843
:1001A000D5280030AD000030AE0029192F14291DCC
:1001B0002F10A9182915A91C2911061BE02829119F
:1001C000291DF728003031020319ED28A00020096D
:1001D0003105A006A01BF228F628C7303002031C08
:1001E000F228F628B00FF528B10A2911FB280030B3
:1001F000B0000030B1002919AC15291DAC11A918A7
:100200002915A91C2911051906292911A91F092930
:100210002911AC190C2929112919AF14291DAF1066
:10022000A9182915A91C2911851917292911291976
:100230002F15291D2F11A9182915A91C2911AF1136
:1002400029192F16291D2F12051A27292F12AF1C25
:100250002A292F122F1E2D29AF1529192F16291DD6
:100260002F12AC1B34292F122F1E3729AF15291935
:100270002F16291D2F122F193E292F122F1E41290B
:10028000AF15AF192915AF1D2911291D6129AF1A05
:100290006129AA0F4C29AB0A00302B0203195729F8
:1002A000A00020092B05A006A01B5C295D290130B8
:1002B0002A02031C5C295D2961290030AA00003054
:1002C000AB002919AF16291DAF12A9182915A91CB1
:1002D00029112F132919AF17291DAF13051A7129D9
:1002E000AF13AF1C7429AF13AF1F77292F1729192C
:1002F000AF17291DAF132F197E29AF13AF1F812907
:100300002F172F1B29152F1F291100303302031916
:100310009029A00020093305A006A01B95299C293F
:1003200009303202031C95299C29291D9A29B20FF4
:100330009A29B30A29119D2929152919A917291DB7
:10034000A913A9182915A91C291134102919B414A5
:10035000291DB410851AAD29B410B41CB029341469
:100360002919B414291DB410AC1BB729B410B41C3E
:10037000BA29341434182915341C2911291DC4290B
:100380000030B2000030B300A9182915A91C2911AA
:100390002C18CB29291129190614291D0610A91872
:1003A0002915A91C2911A91BD6292911291DDC29C8
:1003B0000030B5000030B600A9182915A91C291174
:1003C000A91BE329291129198615291D8611A918A8
:1003D0002915A91C2911051BEE2929112919AC176A
:1003E000291DAC13A9182915A91C29113411291983
:1003F000B415291DB4110618FE29B411B41D012A23
:1004000034152919B415291DB4118619082AB411F7
:10041000B41D0B2A341534192915341D2911291935
:100420000616291D0612A9182915A91C29118619B5
:100430001A2A291129198616291D8612A918291583
:10044000A91C2911861A252A2911341A2B2A1D3094
:10045000B7000030B80034162919432A003038029A
:100460000319392AA00020093805A006A01B3E2A3E
:10047000422A1D303702031C3E2A422AB70F412A66
:10048000B80A2915472A0030B7000030B8002919EA
:100490008616291D8612A9182915A91C29110519C6
:1004A000522A291100303A0203195D2AA0002009BE
:1004B0003A05A006A01B622A692A09303902031CEA
:1004C000622A692A291D672AB90F672ABA0A2911DF
:1004D0006A2A291529190617291D0613A91829158D
:1004E000A91C2911AC1B752A2911291D7B2A003052
:0A04F000B9000030BA008A011E288E
:02400E00623F0F
:00000001FF
